:10000000025FEA3200000000000000025D0E000006
:10001000000000320000000000000032000000007C
:100020000000000232880000000000025DFE0000B7
:100030005052343032207665722E3131302E3720D6
:100040004864773A482034303030752032382D30CB
:10005000362D30342031303A343120202843295293
:100060006F6765722053702E4A2E207777772E7235
:100070006F6765722E706C2C2074656C2F666178CA
:10008000202B34382035352032373230313332208E
:100090002843296A502D706C2C204D6F6E61204CC6
:1000A0006973612043452C2049534F393030312C3E
:1000B0002031737420436C617373D320202052204D
:1000C00045205320452054D25052333032204C43E7
:1000D0004420763131302E37002D2D2F2D2D202D1F
:1000E0002D3A2D2D004350523A20004C6F633A2098
:1000F000004C4F433A2000D22020202020202020F6
:100100002020202020202020D200454E545259206B
:10011000202000455849542020202000445554599F
:10012000204558495400494E5445524E414C00D147
:1001300020202020202020202020202020202020BF
:10014000D1435243202020204520722072206F206E
:10015000720020202020200020D1466C617368208E
:10016000435243204572726F722000D3436F6E6614
:100170006967204D656D204572726F7200D3205300
:10018000657276696365204F4E00D32053657276A1
:10019000696365204F464600D2204D415354455275
:1001A000204944203D20203F2000D3536574207413
:1001B000696D652048484D4D202020D200D35365FD
:1001C00074206461746520524D4D44445720D20020
:1001D000D22020202020202020202020202020206D
:1001E00020D2D501055245473A200000D3D5021050
:1001F00044206F2077206E206C206F2061206420C7
:1002000000D120202020202020202020202020205D
:10021000202020D1D5030C50617373776F72643F37
:10022000203A2000D2D50410204163636573732007
:1002300064656E696564202000D2D5051020416395
:1002400063657373206772616E7465642000D1D535
:100250000410204163636573732064656E6965648F
:100260002020D2D50610204E6F204475616C2045A9
:100270006E747279202000D3D509104475616C200A
:10028000456E747279204D6F64652000D1D50A0ADD
:100290002020204572726F72202300202020200031
:1002A000D1D50C1020202041504220526573657436
:1002B0002020202000D2D50E104C696D6974206575
:1002C00078636565646564202000D50F0C4E4F523D
:1002D0004D414C20202020202000D1D5041020208A
:1002E0004143434553532044454E59202020D2D505
:1002F0001010204150422056696F6C6174696F6E16
:10030000202000D1D50D10202020204964656E7476
:10031000204F4B20202020D2D510102041504220C9
:1003200056696F6C6174696F6E202000D2D5111010
:10033000204E6F206F6E6520696E736964652020A2
:1003400000D1D51210202020557365722049442019
:100350003D203F202000D320202020552053204541
:100360002052D2D51610202050726F6772616D6DC9
:10037000696E6700D3202020494E5354414C4C45B0
:100380005220202020D2D51610202050726F677284
:10039000616D6D696E6720202000D22020202046EC
:1003A000205220452045202020202000D22020203F
:1003B0004520582049205320542053202000D1D5D7
:1003C000041020204143434553532044454E5920B7
:1003D0002020D2D506102020496E70757420426C02
:1003E0006F636B73202000D1D5041020204143435C
:1003F0004553532044454E59202020D2D507102084
:1004000020434C4F534544204D4F4445202020006D
:10041000D1D5041020204143434553532044454E39
:1004200059202020D2D508104F7574206F66207493
:10043000696D65207A6F6E6500D1D504102020416A
:1004400043434553532044454E59202020D2D50BD9
:1004500010204F464620636F6E646974696F6E208A
:100460002000D1D51310202053574954434820442D
:10047000454E59202020D2D508104F7574206F6644
:100480002074696D65207A6F6E6500D1D5041020E7
:10049000204143434553532044454E59202020D208
:1004A000D5141020202020505245414C41524D205F
:1004B00020202000D1D5151020537769746368651A
:1004C000722049443D203F2000C28E53890F43894A
:1004D00010758BD6758D97C28FD28E308FFDC28EE0
:1004E00022C28E53890F438910758BEB758DCBC259
:1004F0008FD28E308FFDC28E22C28E53890F4389D8
:1005000010E58AC4242BF58B758DEBC28FD28E300B
:100510008FFDC28E22F9C3137004A253801814C039
:10052000E0030303540F2443F8D0E0540704F5F02C
:10053000E213D5F0FCE992E02275F0061205E922FB
:10054000C2A075F0061205E9D2A0221205401205DC
:1005500039120540120539120540120539120540BD
:1005600012053912054075F0181205E922C2A0756E
:10057000F04B1205E9D2A022755A0412324DC2A0E6
:1005800075F0C81205E9D2A022755A0512324D1233
:10059000056D75F01E1205E912056D22755A0712D8
:1005A000324D12055722755A0612324D12055D2240
:1005B00012054B12054B22755A0712324D755A0619
:1005C00012324D12055D12055D12055D22C2A1C2F7
:1005D0006812054075F0121205E9D2A1C268221214
:1005E000054075F0121205E9221204C9201E07C049
:1005F000F0122482D0F0D5F0F0227004A253B3227E
:10060000C0E014120609D0E022C0E0030303540F37
:1006100028F8D0E0C0E0540704F5F0E213D5F0FC70
:10062000D0E02212054B75F0641204C9D5F0FA220D
:1006300012055775F0C81204C9D5F0FA80F22230BD
:100640001716C217C2AC1204F91204F9D299120794
:1006500025C260D2B6125E09301116C211C2AC12A8
:1006600004F91204F9D299121458C260D2B6125E7B
:1006700009301316C213C2AC1204F91204F9D2994C
:100680001214DDC260D2B6125E09301216C212C256
:10069000AC1204F91204F9D299121379C260D2B6DD
:1006A000125E09301416C214C2AC1204F91204F915
:1006B000D2991213BBC260D2B6125E09301516C2AF
:1006C00015C2AC1204F91204F9D299121525C260B0
:1006D000D2B6125E09301616C216C2AC1204F91256
:1006E00004F9D2991215B8C260D2B6125E09301858
:1006F00016C218C2AC1204F91204F9D299125A9116
:10070000C260D2B6125E09E57A6013B40105122CFC
:10071000928008B40205122CA18000757A00122480
:100720008212595C22125C64C2B6753700740312DF
:100730003E98E51E123E98E51F123E987450123EF8
:1007400098747D123E98900000E535600F9003E8A4
:100750001460099007D0146003900BB87E7D7F0869
:1007600075F000C0F0125C5FB40203D38001C3D007
:10077000E033F5F0A3DFEC123E98DEE2E537123EFF
:10078000983099FD22C0F075F0DCD5F005B2B512B5
:1007900055FFC0F01209CFD0F030E7EED0F022AA1A
:1007A000F0120785E532652FF5F0E533653045F049
:1007B000600C1208F6852F32853033120785120936
:1007C000941207851209BC1207851209038AF022C8
:1007D000AAF0120785E532652FF5F0E5336530455F
:1007E000F0600C1208F6852F32853033120785121F
:1007F00009801207851209BC1207851209038AF0C5
:10080000227920752F017530037531E09000811237
:1008100007851208F61207851209547900752F0111
:100820007530047531009000A11207851208F61288
:10083000078512095479E0752F017530057531006F
:100840009001A11207851208F61207851209548536
:100850002F3285303322AAF0120785E532652FF555
:10086000F0E533653045F0600C1208F6852F3285CF
:10087000303312078512093C8AF022AAF01207854C
:10088000E532652FF5F0E533653045F0600C120870
:10089000F6852F328530331207851209248AF0221B
:1008A000C0F075F00833C297928300D297D5F0F567
:1008B000D0F022C0F075F008C297D29700A2823320
:1008C000D5F0F5D0F022D2B7D297D283D282D2849B
:1008D00022E53033E52F3322C3E5303322E53122E0
:1008E0001208A01208D11208A01208D81208A012EB
:1008F00008DD1208A0221208C6C28474531208E050
:10090000D284221208C6C28474581208E0D284220B
:100910001208C6C28474541208E0E41208A0120837
:10092000B3D284221208C6C28474541208E0E412BE
:1009300008A01208B3F608D9F9D284221208C6C258
:100940008474541208E0E41208A01208B3F208D923
:10095000F9D284221208C6C28474541208E0E41248
:1009600008A01208B3F0A3D9F9D284221208C6C095
:10097000E0C28474841208E0D0E01208A0D284227D
:100980001208C6C28474841208E0E61208A008D9CE
:10099000F9D284221208C6C28474841208E0E212DA
:1009A00008A008D9F9D284221208C6C2847484121D
:1009B00008E0E01208A0A3D9F9D284221208C6C226
:1009C0008474831208E0D2841204C91204C922C2BA
:1009D0008474571208A01208B3D28422D283D28220
:1009E000D297D2B7D284B2B575F0021204C9D5F04D
:1009F000FAC2B7B2B575F0021204C9D5F0FAD2B78F
:100A0000B2B522752F017530DB75310012078512E2
:100A10000C9E7532FF7533FF22AE83AD8290DB00F2
:100A20007F207404F9747CF8752F018583308582EA
:100A30003112087B787CE66E702508E66D70200820
:100A4000E6601AB4FF028013167404F9747CF8751A
:100A50002F018583308582311207D0C322D322A390
:100A6000A3A3A3DFBD80F490DB007F207404F9749E
:100A70007CF8752F0185833085823112087B787C64
:100A8000E66E700908E66D700408E6FC22A3A3A3D5
:100A9000A3DF0A7CFF2290DB007F207BFF7404F938
:100AA000747CF8752F0185833085823112087B783C
:100AB0007CE66E702C08E66D702708ECB4FF0D78AC
:100AC0007C76FF0876FF0876FF0874FFF67404F959
:100AD000747CF8752F018583308582311207D0C36D
:100AE00022BBFF10787CE6B4FF0A08E6B4FF05C31A
:100AF00074209FFBA3A3A3A3DFA3BBFF02D322EB1E
:100B0000232354FC2400F5827583DB50020583788F
:100B10007CEEF608EDF608ECF608E4F67404F974D9
:100B20007CF8752F018583308582311207D0C3226E
:100B300075830075F08E752F02858330753100C086
:100B4000F0C083120785120C9ED0830583D0F0D5A8
:100B5000F0E475830075F0DA752F03858330753105
:100B600000C0F0C083120785120C9ED0830583D08D
:100B7000F0D5F0E47532FF7533FF2275830075827E
:100B80000075F08EC0F0C082C083752F028583305F
:100B90007531001207851208F6D083D082C082C05A
:100BA00083752F008582307531001207851209BCCC
:100BB000D083D08205830582D0F0D5F0C77583003D
:100BC00075820075F0DAC0F0C082C083752F03858E
:100BD00083307531001207851208F6D083D082C0A9
:100BE00082C083752F01858230753100120785120E
:100BF00009BCD083D08205830582D0F0D5F0C775BB
:100C000032FF7533FF2275830075820075F08EC048
:100C1000F0C082C083752F008583307531001207C4
:100C2000851208F6D083D082C082C083752F0285DA
:100C300082307531001207851209BCD083D082053D
:100C4000830582D0F0D5F0C775830075820075F0FA
:100C5000DAC0F0C082C083752F0185833075310002
:100C60001207851208F6D083D082C082C083752F08
:100C7000038582307531001207851209BCD083D0FC
:100C80008205830582D0F0D5F0C77532FF7533FF3A
:100C9000221208C6C28474501208E0D284221208BC
:100CA000C6C28474811208E0D284221208C6C284AB
:100CB00074841208E0E81208A0D9FAD28422AAF0BB
:100CC000120785E532652FF5F0E533653045F060B4
:100CD0000C1208F6852F32853033120785120CABC3
:100CE0001207851209BC8AF0221208C6C284745405
:100CF0001208E0E41208A0E4C0E01208B3D0F02526
:100D0000F0D9F5D28422758300758202800675833E
:100D100000758200E475F08D85822F8583307531F2
:100D200000C082C083C0F0C0E01207851208F6122E
:100D300007857900120CE9D0F025F0D0F0D083D0EF
:100D4000820583D5F0D285822F858330753100C02E
:100D5000E01207851208F61207857920120CE9D0F7
:100D6000F025F07532FF7533FF227583007582031D
:100D70008006758300758201E475F0DA85822F851F
:100D80008330753100C082C083C0F0C0E012078597
:100D90001208F61207857900120CE9D0F025F0D080
:100DA000F0D083D0820583D5F0D27532FF7533FF42
:100DB00005E02275830075F000752F00858330757E
:100DC0003100C0F0C083120785120C9ED0830583CA
:100DD000D0F0D5F0E47532FF7533FF75830075F000
:100DE000DA752F01858330753100C0F0C08312079A
:100DF00085120C9ED0830583D0F0D5F0E47532FFC8
:100E00007533FF221205637555FA3090FA75F005B7
:100E10001204C9D5F0FA7555FA2090FA22E577B494
:100E200006FAE583125316E5821253167800E21291
:100E300053167801E21253167802E2125316120E7C
:100E40000422C0E0E577B40928D0E0787CE61253AC
:100E50001608E612531608E612531608E612531641
:100E600008E612531608E6125316D2AF120E04C04B
:100E7000E0D0E022E577B4053DED600F1414600B7F
:100E8000146008146005ED2488502BE583C082129D
:100E90005316D082E582125316ED125316787CE673
:100EA00012531608E612531608E612531608E612F5
:100EB000531608120E042222E577B405F9ED2488B2
:100EC00050F4C082C083787CE60354012430E612DB
:100ED000531608E6125316D083D082E583C082C031
:100EE00083125316D083D082E582C082C08312530E
:100EF00016120E04D083D0822222E577B4050FEDBE
:100F00002488500A74303073027431120E04223077
:100F100008597881E6540FC0E0E6C4540375F00A1E
:100F2000A4D0F025F0FD7882E630E402240A540FC4
:100F3000FE901A007F3C7404F97400F8752F018547
:100F400083308582311208567800E26D701708E20E
:100F50006E701208E2C42354E0F5F07882E6541F64
:100F600045F0F68006A3A3A3A3DFCB2212620312EF
:100F70000F0F126212FEAFF012574C7DFF0DED30D5
:100F8000E70122D27375F004A42481F582E5F034E0
:100F900000F583C082C083787CE0F6A308E0F6A366
:100FA00008E0F6A308E0F6D083D082120E74787CB5
:100FB0008683088682787CB6FF0708B6FF03021096
:100FC00025C3E58233F582E58333F583E58224E0AA
:100FD000F582E5833405F583787EE6704808E6609F
:100FE00044FB7402F9747CF8752F01858330858287
:100FF0003112087B120EB7A3A3787CE60856B4FF23
:1010000003021025787C86F053F07F08E6C39EC06B
:10101000E0E5F09FD0F0400445F07009787CE6A24E
:10102000E79273DBBD120EF9BD003DB273122C20A6
:101030004033203C30201F0E303D0B2052053073D2
:1010400024800320731FA273925292E0A25392E174
:10105000F5F013925365F030E00B205305122CB0DD
:101060008003122CBF020F7DED14C0E00303035474
:101070000F2443F8D0E0540704FB7400D333DBFDA6
:10108000307305FBE24B8004F4FBE25BF2020F7D60
:101090001208A01208D11208A01208D8D2E0120833
:1010A000A01208DD1208A0221208C6C284745412CD
:1010B0001090E41208A01208B3F608D9F9D28422DD
:1010C0001208C6C2847484121090E61208A008D9CF
:1010D000F9D2842290FC00752F0475300075310020
:1010E000C082C0837555FA1207851208F6852F79DC
:1010F0008530787908787C1207851210A81212D0F2
:10110000D083D0827044C082C08378808683088672
:10111000821211814024787E868308868212118192
:1011200040181211A0E582600AE575B5780CE576E5
:10113000B57907D083D08202115C787EE6249AF6D6
:101140001213131252BCD083D0820530E5307002E6
:10115000052FA3E582458370871211637532FF75F1
:1011600033FF22787E760008760078807600087655
:10117000000876000876007579047578001212EF81
:1011800022C082C083E5822400F582E5833480F5A5
:10119000834005D083D08222D083D0829000002269
:1011A000E58275F008A4F582E5F0C58375F008A422
:1011B0002583F583E5F03404F576E5822400F58295
:1011C000E5833400F583500205768583752212523B
:1011D000CCD083D08222C082C0831212A970EF7853
:1011E0007E868308868212118140E31211A01216B6
:1011F0001D787C76007880E518F608E519F6087603
:10120000000876007408F9747CF885762F858330A1
:101210008582311207D07404F97480F885762F85A1
:10122000833085823112087B75F004787C7980E602
:1012300067600280990809D5F0F51212B0787E86B1
:1012400083088682A3121181787EA68308A68278FD
:10125000808683088682121181787EE66583700A13
:1012600008E665827004A31211817880A68308A61F
:1012700082C079C0788576798575781212EFD0E0D2
:10128000D0F0B57809C5F0B579028018C5F0C079FD
:10129000C07885F079F578787EE62499F6121313F4
:1012A000D078D079D083D082221212B01212D022FC
:1012B00085792F8578307531001207851208F67907
:1012C00008787C1207851210A8852F3285303322CA
:1012D0007881E618261826182618245566700F7887
:1012E00081E61866186618661866186499662212F0
:1012F00012F6121313227881E618261826182618DB
:101300002455F67881E6186618661866186618641B
:1013100099F62285792F857830753100120785126C
:1013200008F61207857908787C1210C0120785121A
:1013300009BC120785120903852F3285303322122A
:1013400012A97030787EE6C0E008E6C0E008868327
:10135000088682C3D0E09582F582D0E09583F5833C
:1013600050104582600CE5822400F582E5833480CC
:10137000F583C322900000D322C2B612133FE43398
:10138000C0E07537007403123E98E51E123E98E5E2
:101390001F123E987453123E98D0E0123E9874008B
:1013A000123E987400123E98E583123E98E5821230
:1013B0003E98E537123E983099FD22C2B6E5356079
:1013C00004F4FF8004FF1211637537007403123EAA
:1013D00098E51E123E98E51F123E987456123E98EC
:1013E000EF123E98E537123E983099FD227401C005
:1013F000E0787C75F008E4F608D5F0FBD0E0D32265
:1014000012133F40E860E8788086830886821214D1
:1014100013C322C082C083E58275F008A4F582E57B
:10142000F0C58375F008A42583F583E5F03404F551
:1014300076E5822400F582E5833400F583500205C9
:10144000767408F9747CF885762F8583308582312F
:1014500012087BD083D0822212133F7F08500512DE
:1014600011637F00787E8663088664088665088637
:1014700066C2B67537007403123E98E51E123E9898
:10148000E51F123E987454123E98E535123E98EFCF
:10149000123E98E535603CE5666564F5F0E5656506
:1014A0006345F0600B8566828565831214138003A3
:1014B0001213EF856682856583A31211818582668A
:1014C000858365787C75F008E6123E9808D5F0F8BB
:1014D000D535C4E537123E983099FDC322E5357005
:1014E00007C2AF12133F5005E535F4800C7880A693
:1014F0006508A6661212EFE535D2AFC0E0C2B67538
:1015000037007403123E98E51E123E98E51F123E06
:10151000987455123E98D0E0123E98E537123E98E6
:101520003099FDD322C2B6126203753700740312DC
:101530003E98E51E123E98E51F123E987457123EE3
:10154000987881E623235403123E987882E630E4AB
:1015500002240A541F123E987881E6C45401F5F023
:10156000A4E5F0E6540F25F0123E987881E6C454C5
:1015700001F5F0A4E5F0E6540F25F0123E98787FCF
:10158000E6C45403F5F0A4E5F0E6540F25F0123E4E
:1015900098787EE6C45403F5F0A4E5F0E6540F25F0
:1015A000F0123E987882E603C45407123E98E5375D
:1015B000123E983099FDD322C2B6753700740312DB
:1015C0003E98E51E123E98E51F123E987458123E52
:1015D000987420232354FC04123E987420123E98E1
:1015E00090DB007F207404F9747CF8752F018583EB
:1015F0003085823112087B787CE6123E9808E6122C
:101600003E9808E6123E9808E6123E9808A3A3A367
:10161000A3DFD2E537123E983099FDD32212620340
:101620007882E630E402240A540FC4F97881E6C4D3
:10163000540375F00AA4F5F0E6540F25F0C31349DE
:10164000787DF67881E692E754C0F9787FE6C45455
:101650000775F00AA4F5F0E6540F25F049F97880F3
:10166000E6C4540375F00AA4F5F0E6540F25F0F52E
:10167000F0787EE654702345F0787FF6787EE9F6C0
:1016800022C082C083E52F125316E530125316781C
:101690007EE612531608E612531608E61253160891
:1016A000E6125316120E04D083D0822253620F53D7
:1016B000610F5318F053190FC2AFE5612324ADF841
:1016C000E5184519F608A61A056153610FE561B5DD
:1016D0006205056253620FD2AFC3E56195625002A5
:1016E000241024F45003756E0022E562B561057480
:1016F00000780022C33324ADF8E6C0E008E6F8D055
:10170000E022223054FDC2A075F0061205E9D2A0F5
:1017100075F0141205E9E545C25422301E037554D4
:10172000F01222B8205407740F301E0580F31217F0
:101730000322F5F00303543FB40267E53E640860FA
:1017400005E53EB40D59E5F089F0C0F030081CC045
:10175000E07877E26013C3335005D0E002177E12C1
:10176000051550F6D0E002176BD0E0D0F0A9F05488
:1017700003B40211C231A231B392A5021871D0F0A4
:10178000A9F0021871B4010AD231A231B392A502B4
:101790001871B4030AB231A231B392A502187102D2
:1017A000186FB40365E53F64086005E53FB40DEFCD
:1017B000E5F089F0C0F030081CC0E07878E26013F2
:1017C000C3335005D0E00217E812051550F6D0E0FB
:1017D0000217D5D0E0D0F0A9F05403B40211C23200
:1017E000A232B392A6021871D0F0A9F0021871B417
:1017F000010AD232A232B392A6021871B40309B21E
:1018000032A232B392A680698065B40462E5406476
:10181000086005E540B40D57E5F089F0C0F03008E8
:101820001CC0E0787EE26013C3335005D0E002189C
:101830004F12051550F6D0E002183DD0E0D0F0A9C7
:10184000F05403B4020FC237A237B392808022D083
:10185000F0A9F0801CB40109D237A237B39280807E
:1018600010B40309B237A237B3928080048000D34A
:1018700022C322787375F00EE4F208D5F0FB74FFF2
:10188000787BF2787CF222D24E6F20657874656E98
:10189000646564202020202020202000756FFF1226
:1018A0001873C208C207120D72602E20082A740134
:1018B000F9747CF8752F0075308C7531EE12087B49
:1018C000797CE7B4FF12C246C247C248C249C24A45
:1018D000C24BC24CC24DC24E221208017401F974AF
:1018E0006FF8752F017530037531A012087B740EE7
:1018F000F97473F8752F017530037531A11208560C
:101900007410F97453F8752F017530037531C012D6
:1019100008567410F97463F8752F0175300375312A
:10192000D0120856D208D20722797C774809774E20
:1019300009776E0977A07404F9747CF8752F007527
:10194000308D7531201207D07404F9747CF8752F2E
:101950000275308D7531201207D022E4A22492E066
:10196000A22592E1A22692E2797CF77401F9747CB7
:10197000F8752F0075308C7531E81207D02274018C
:10198000F9747CF8752F0075308C7531E812087B7E
:10199000797CE7A2E09224A2E19225A2E29226229B
:1019A000797CE4A23892E0A23992E1A23A92E2A2D2
:1019B0001C92E392E492E5A23C92E6A23D92E7F704
:1019C00009E4A23B92E0A23E92E1A23F92E2A24051
:1019D00092E3A24292E4A24392E5A24492E6A24597
:1019E00092E7F709E4A24692E0A24792E1A2489268
:1019F000E2A24992E3A24A92E4A24B92E5A24C925F
:101A0000E6A24D92E7F7E4A24E92E0A20292E1A292
:101A10000392E2F77404F9747CF8752F0075308C2A
:101A20007531EC1207D0227404F9747CF8752F001C
:101A300075308C7531EC12087B797CE7A2E0923826
:101A4000A2E19239A2E2923AA2E3921CA2E6923C6F
:101A5000A2E7923D09E7A2E0923BA2E1923EA2E218
:101A6000923FA2E39240A2E49242A2E59243A2E610
:101A70009244A2E7924509E7A2E09246A2E192478A
:101A8000A2E29248A2E39249A2E4924AA2E5924BD2
:101A9000A2E6924CA2E7924D09E7A2E0924EA2E1A3
:101AA0009202A2E2920322797CF77401F9747CF825
:101AB000752F0075308C7531E41207D0227401F94E
:101AC000747CF8752F0075308C7531E412087B79C1
:101AD0007CE7227401F97438F8752F0075308C7525
:101AE00031FC1207D0227401F97438F8752F007593
:101AF000308C7531FC12087B227401F97439F87549
:101B00002F0075308D7531001207D0227401F974E1
:101B100039F8752F0075308D75310012087B2274ED
:101B200002F9743FF8752F0075308C7531FD12087D
:101B3000567402F97441F8752F0075308D753101B6
:101B4000120856227402F9743FF8752F0075308C14
:101B50007531FD12079F7402F97441F8752F0075F5
:101B6000308D75310112079F227401F9743AF875AE
:101B70002F0075308C7531F01207D07401F9743B69
:101B8000F8752F0075308C7531F41207D07401F997
:101B9000743CF8752F0075308C7531F61207D074CF
:101BA00001F9743DF8752F0075308C7531F212070C
:101BB000D0227401F9743AF8752F0075308C7531A4
:101BC000F012087B7401F9743BF8752F0075308CA6
:101BD0007531F412087B7401F9743CF8752F0075A7
:101BE000308C7531F612087B7401F9743DF8752F4D
:101BF0000075308C7531F212087B227401F9743E45
:101C0000F8752F0075308C7531F81207D07401F912
:101C1000743FF8752F0075308C7531FA1207D07447
:101C200001F97440F8752F0075308C7531FB12077F
:101C3000D0227401F9743EF8752F0075308C75311F
:101C4000F812087B7401F9743FF8752F0075308C19
:101C50007531FA12087B7401F97440F8752F00751C
:101C6000308C7531FB12087B227402F9741EF875F2
:101C70002F0075308C7531E01207D0227402F97490
:101C80001EF8752F0075308C7531E012087B22C06C
:101C900082C083E58275F008A42420F582500205F5
:101CA000F0A8F0E58375F008A4282400F583787C7B
:101CB00076FF7401F9747CF8752F00858330858276
:101CC000311207D0A3A3A3A3A37401F9747CF87500
:101CD0002F008583308582311207D0D083D082C215
:101CE00007220809E7C4F5F066540F700D08E7F500
:101CF000F066540F7004DAEAE422E6540FC5F0549B
:101D00000FC395F09206740122788179277A03E651
:101D1000C4540FF309E6540FF30908DAF27927786F
:101D2000A07A06E6540FF6E36670080908DAF4E4D0
:101D3000C25A22792C78A57A06C3E3961918DAFAE2
:101D40009206792C78A57A06E3540FB40F08E6546E
:101D50000FB40F108008E6540FB40F0B800618194B
:101D6000DAE680CB740122C3E396B4090280121430
:101D7000600FC3E3F5F0E695F0B409028003147038
:101D8000E3E9B42704E4D25A221918E366540F6039
:101D9000F080D1121D09701A305A17203B157518A2
:101DA0005085831985821A1216AC7553B4D256D257
:101DB00059E42204227408F9747CF8752F007530F8
:101DC0008C7531C012087B7894797C7A05121CE4FA
:101DD000227408F9747CF8752F0075308C7531C049
:101DE00012087B121D93227405F9747CF8752F007C
:101DF00075308C7531C01207D0227403F97481F8E4
:101E0000752F0075308C7531C51207D022C082C085
:101E100083E5822420F582E583347DF5837401F91E
:101E20007441F8752F0085833085823112087BD08C
:101E300083D082C082C083E58275F008A42420F597
:101E400082500205F0A8F0E58375F008A42824006C
:101E5000F5837408F9747CF8752F008583308582CA
:101E60003112087BD083D08222C082C083E5827584
:101E7000F008A42420F582500205F0A8F0E583754F
:101E8000F008A4282400F5837408F97494F8752FD9
:101E90000085833085823112087BD083D08222C0B6
:101EA00082C083E58275F008A42420F582500205E3
:101EB000F0A8F0E58375F008A4282400F5837406E3
:101EC000F9747CF8752F0085833085823112087B88
:101ED000D083D082227405F9747CF8752F00753098
:101EE0000075312012087B7894797C7A05121CE405
:101EF00022751B20751C009000007405F9747CF895
:101F0000752F00851C30851B3112087B7894797CF5
:101F10007A05121CE46018E51B2408F51B50020525
:101F20001CA3E583B40FD3E582B4A0CE74012212C2
:101F30001E0DE42220070280B8751B00751C007579
:101F4000739F75740FE573251BC2E0F582E5743548
:101F50001CF583C082C083E5822400F582E58334CA
:101F60001BF5837402F9747CF8752F018583308525
:101F7000823112087B787C8683088682121E0D7857
:101F800094797C7A05121CE47005D0F0D0F022D050
:101F900083D082C3E58313F583E58213F58220069F
:101FA00014E58245836023E58224FFF573E58334DD
:101FB000FFF5748007A385821B85831CC3E5739599
:101FC0001BE574951C4003021F45740122751B25F7
:101FD000751C009000007403F97481F8752F00855A
:101FE0001C30851B3112087B121D936018E51B24E1
:101FF00008F51B5002051CA3E583B40FD9E582B494
:10200000A0D4740122121E0DE42278A0E6540FB46D
:102010000F030220A420070280B3751B00751C006B
:1020200075739F75740FE573251BC2E0F582E57427
:10203000351CF583C082C083E5822400F582E583E8
:10204000343BF5837402F9747CF8752F0185833075
:1020500085823112087B787C8683088682121E0D69
:10206000121D937005D0F0D0F022D083D082C3E54A
:102070008313F583E58213F582200614E5824583F8
:102080006022E58224FFF573E58334FFF574800751
:10209000A385821B85831CC3E573951BE574951C82
:1020A0004002808274012278947A0579A8E6540F60
:1020B000C4F5F008E6540F45F0F70809DAEF22C23C
:1020C000A3C266C2A2C269C2A1C268D2B775F00239
:1020D0001204C9D5F0FA20B72BD21ED2A3C266C211
:1020E000A2D269D2A1C268D2A4C267120563B2B5F6
:1020F00075F00F1204C9D5F0FA30B7EF122178C28B
:10210000AF025FA3D2A0120D0E700712213F12186A
:102110009C22C21E7555FA75F0641204C9D5F0FAF6
:10212000C2A0C2A2C26975F0641204C9D5F0FAD285
:10213000A0D2A2C269D2B71204E130B79C80D312F8
:10214000197E121A27121ABDA2E0924FA2E19250F4
:10215000A2E29251121AE6121B0C121BB2121C328E
:10216000121B1F121C7C22C2A3C266C2A2C269C279
:10217000A1C268D2A4C26722D21E12517F40E8C217
:10218000A3C266C2A2C269C2A1C268D2A4C267C009
:102190001EC01F787C9000007A08E6F008A3DAFAE7
:1021A0001221CD787C9000007A08E0F608A3DAFAD4
:1021B000900000124B8D121DE7121DFAD01FD01E89
:1021C000121C69124C07121163120A0322120DB37A
:1021D000751E30751F30C224C225C226C238C239CE
:1021E000C23AC21CC23CC23DC23BD23EC23FC24008
:1021F000C242C243C244C245C246C247C248C249A3
:10220000C24AC24BC24CC24DC24E783F7422F20841
:102210007400F278417406F2087400F2C24FC250A2
:10222000C251753804753909753A01753B02753C20
:1022300004753D04753E07753F00754000121C692A
:1022400012195B1219A0C2E0A24F92E0A25092E1D3
:10225000A25192E2121AA7121AD3121AF9121B698A
:10226000121BFB121B44C208C207121929125B4A37
:1022700022306B04C26B800975F00C20B205D5F0DA
:10228000FAD322C322122271502DE8C0E0E9C0E047
:10229000EAC0E0755A0075F0031204C9D5F0FA12CD
:1022A00030DE75F0031204C9D5F0FA122F62D0E0C7
:1022B000FAD0E0F9D0E0F822D2638008C26312239A
:1022C0002A754200C21DD26B7555FA7440301E0249
:1022D000740CF552C262C254E55260391222852054
:1022E000623375F0031204C9D5F0FA12063F201EBE
:1022F00003201D183054E120631B75526012170330
:10230000B40B0D75F0081204C9D5F0FAD26280053D
:1023100012231D80C3C261D2AF7555FA2253420702
:10232000F8E54224A0C8F605422278A075F00874AA
:10233000FFF608D5F0FB22306109202303D22322C7
:10234000C26122C22322D2638004D26BC263C21D47
:102350007555FAD2227440301E02740CF5521223C5
:102360002A754200C262C261C254C26512063F2091
:102370001E03201D2112228520621D20611A305467
:1023800021206314755260121703B40B1275F00804
:102390001204C9D5F0FAD2627555FA12574C2212BE
:1023A000231DE55260F212574C3065FD80BC853824
:1023B00056755700B230E5386002D230A230B39281
:1023C000A7D26B22301D012278A0760A08760380FE
:1023D0000778A0760A0876010875F06484F608E5A7
:1023E000F075F00A84F608A6F0754205D21D227534
:1023F00018C0751900751A011216AC22755100C269
:10240000587518C0751900751A021216AC22D256EA
:102410007553B475185075190F751AFF1216AC2242
:10242000C20A1223AE20480C75181075190F751AC0
:10243000FF1216AC2220480C75182075190F751A5A
:10244000FF1216AC2275186075190F751AFF121657
:10245000AC2275187075190F751AFF1216AC22127E
:102460005B4A7518C0751900751A0E1216AC221247
:1024700025C6400D1227C240081229724003122BB4
:102480005522301E03C38006A290302401B3783653
:10249000E233F2B4FF0280060225D002267C202718
:1024A00003202DF7D22D30081CC0E07873E26013B2
:1024B000C3335005D0E002267C12051550F6D0E05B
:1024C0000224C5D0E0E53A60D2B40126D20B122333
:1024D000EF30301520460C755702755602304A030E
:1024E00075560185395102267C20440312240E02C0
:1024F000267CB40215303903205309206D061224BE
:102500002002266E12243502267CB40308C2531220
:10251000244502267CB40705D277757B03B4090CE9
:102520002053032045030225B802267CB40A027416
:102530003DB4340874001223C402267CB4350874F8
:10254000101223C402267CB4360874111223C4026C
:10255000267CB4370874201223C402267CB4381BAE
:102560007401F9747CF8752F0075308C7531F11297
:10257000087B787CE61223C402267CB4391B7401E4
:10258000F9747CF8752F0075308C7531F112087B69
:10259000787CE61223D102267CB43C0612245F022A
:1025A000266EB43D13205308D25312245202266ED5
:1025B000C25312244502266E751890751909F51A32
:1025C0001216AC02267CE53AB40B03A22D22C322DC
:1025D00070F1202703302DEBC22D30081CC0E078AD
:1025E00073E26013C3335005D0E002267C12051558
:1025F00050F6D0E00225F9D0E0E53A6022B40107B8
:10260000C20B1223FC8075B402028070B40307D29F
:10261000531224528066B409082053443045418047
:102620005BB40A02743DB432028051B43302804C70
:10263000B4340302267CB4350302267CB43603028C
:10264000267CB4370302267CB4380302267CB439D6
:102650000302267CB43C0302267CB43D0302267CA4
:102660007518A0751909F51A1216AC02267C10040B
:102670000302267C1257A712059CD204C227301EE3
:1026800003C38006A291302501B37837E233F2B458
:10269000FF0280060227CC022878202803202EF78C
:1026A000D22E30081CC0E07874E26013C3335005AA
:1026B000D0E002287812051550F6D0E00226C1D0ED
:1026C000E0E53B60D2B40126D20B1223EF30301587
:1026D00020460C755702755602304A03755601851F
:1026E000395102287820440312240E022878B402BB
:1026F00015303903205309206D0612242002286A60
:10270000122435022878B40308C253122445022843
:1027100078B40705D277757B03B4090C20530320E6
:1027200045030227B4022878B40A02743DB4340881
:1027300074001223C4022878B4350874101223C41C
:10274000022878B4360874111223C4022878B437EA
:102750000874201223C4022878B4381B7401F97459
:102760007CF8752F0075308C7531F512087B787CFC
:10277000E61223C4022878B4391B7401F9747CF87A
:10278000752F0075308C7531F512087B787CE61258
:1027900023D1022878B43C0612245F02286AB43D93
:1027A00013205308D25312245202286AC25312240F
:1027B0004502286A75189075190AF51A1216AC02A6
:1027C0002878E53BB40B03A22E22C32270F1202807
:1027D00003302EEBC22E30081CC0E07874E2601388
:1027E000C3335005D0E002287812051550F6D0E02A
:1027F0000227F5D0E0E53B6022B40107C20B1223AB
:10280000FC8075B402028070B40307D253122452C4
:102810008066B40908205344304541805BB40A0205
:10282000743DB432028051B43302804CB43403029C
:102830002878B43503022878B43603022878B437F0
:1028400003022878B43803022878B43903022878C0
:10285000B43C03022878B43D030228787518A075AB
:10286000190AF51A1216AC02287810040302287807
:102870001257A712059CD204C228301E03C380063B
:10288000A292302601B37838E233F2B4FF02800618
:1028900002297C022A0F202903202FF7D22F30088B
:1028A0001CC0E07875E26013C3335005D0E0022A03
:1028B0000F12051550F6D0E00228BDD0E0E53C60CF
:1028C000D2B40705D277757B03B4090C20530320DB
:1028D0004503022964022A0FB40A02743DB4340885
:1028E00074001223C4022A0FB4350874101223C4D2
:1028F000022A0FB4360874111223C4022A0FB43707
:102900000874201223C4022A0FB4381B7401F9740E
:102910007CF8752F0075308C7531F712087B787C48
:10292000E61223C4022A0FB4391B7401F9747CF82F
:10293000752F0075308C7531F712087B787CE612A4
:1029400023D1022A0FB43C0612245F022A01B43DAF
:1029500013205308D253122452022A01C2531224C4
:1029600045022A0175189075190CF51A1216AC0259
:102970002A0FE53CB40B03A22F22C32270F12029B9
:1029800003302FEBC22F30081CC0E07875E26013D3
:10299000C3335005D0E0022A0F12051550F6D0E0DF
:1029A0000229A5D0E0E53C6009B409082053443071
:1029B0004541805BB40A02743DB432028051B433A5
:1029C00002804CB43403022A0FB43503022A0FB438
:1029D0003603022A0FB43703022A0FB43803022A3F
:1029E0000FB43903022A0FB43C03022A0FB43D038B
:1029F000022A0F7518A075190CF51A1216AC022AC6
:102A00000F100403022A0F1257A712059CD204C20A
:102A100029301E03C38006A285303301B37839E222
:102A200033F2B4FF028006022B5F022C0B2034032A
:102A30002036F7D23630081CC0E0787DE26013C340
:102A4000335005D0E0022C0B12051550F6D0E002F1
:102A50002A54D0E0E53D60D2B40126D20B1223EF18
:102A600030301520460C755702755602304A0375F2
:102A70005601853951022C0B20440312240E022CDE
:102A80000BB40215303903205309206D061224209F
:102A9000022BFD122435022C0BB40308C25312245E
:102AA00045022C0BB40705D277757B03B4090C20C3
:102AB0005303204503022B47022C0BB40A02743D3A
:102AC000B4340874001223C4022C0BB435087410FB
:102AD0001223C4022C0BB4360874111223C4022C26
:102AE0000BB4370874201223C4022C0BB4381B74A7
:102AF00001F9747CF8752F0075308C7531F312086C
:102B00007B787CE61223C4022C0BB4391B7401F9C8
:102B1000747CF8752F0075308C7531F312087B7852
:102B20007CE61223D1022C0BB43C0612245F022B4C
:102B3000FDB43D13205308D253122452022BFDC280
:102B400053122445022BFD75189075190DF51A12B4
:102B500016AC022C0BE53DB40B03A23622C3227047
:102B6000F12034033036EBC23630081CC0E0787DEB
:102B7000E26013C3335005D0E0022C0B1205155050
:102B8000F6D0E0022B88D0E0E53D6022B40107C218
:102B90000B1223FC8075B402028070B40307D25379
:102BA0001224528066B40908205344304541805BAA
:102BB000B40A02743DB432028051B43302804CB482
:102BC0003403022C0BB43503022C0BB43603022C55
:102BD0000BB43703022C0BB43803022C0BB43903AB
:102BE000022C0BB43C03022C0BB43D03022C0B75DE
:102BF00018A075190DF51A1216AC022C0B1004034F
:102C0000022C0B1257A712059CD204C234205B0180
:102C100022C25B751840751900751A001216AC2295
:102C2000E53A64036008E53B64036002C322D322F3
:102C30001205DF30080C125398400390FFF1125335
:102C4000DD22C05B122C60D05B2230081312539837
:102C5000400390FFF11253DD5005F55B125434220E
:102C6000E55B7005755B108023B41005755B118002
:102C70001BB41105755B208013B42005755BFF80C4
:102C80000BB4FF05755B008003755BFF12549BE579
:102C90005B22C25375186075190F751AFA1216ACBB
:102CA00022D25375187075190F751AFA1216AC22C4
:102CB000C25375186075190F751AE01216AC22D23E
:102CC0005375187075190F751AE01216AC22122D73
:102CD000C2122E59122EF022122DCF122E66122E53
:102CE000FD22B20C30081CC0E07877E26013C333D9
:102CF0005005D0E0022D4512051550F6D0E0022D0A
:102D000003D0E0E53E604C24F84005E53E022D5E30
:102D1000E53EB40904A209803DB40A04A20B803642
:102D2000B40C03D38030B40D0B302B03022DDCD256
:102D30002BD38022B40E04A20A801BB40F04A27706
:102D40008014022DDCB40D06202B03022DDCC22BD7
:102D5000C38003A253B39231B392A5022DDC300C91
:102D60005E5359037859A2E282564030A2E082575E
:102D70004012A2E182584018C231A231B392A57626
:102D800000022DDCB60102801D76017558408016C8
:102D9000B60202801176027558A0800AB60302803E
:102DA0000576037558CCE55823F55820E00AC23162
:102DB000A231B392A5022DDCD231A231B392A50289
:102DC0002DDCE53EB40B07D231A231B392A522E54A
:102DD0003EB40B07C231A231B392A52230081CC009
:102DE000E07878E26013C3335005D0E0022E3D1244
:102DF000051550F6D0E0022DFBD0E0E53F604C24F5
:102E0000F84005E53F022E56E53FB40904A20980CB
:102E10003DB40A04A20B8036B40C03D38030B40D49
:102E20000B302C03022E73D22CD38022B40E04A2BA
:102E30000A801BB40F04A2778014022E73B40D060F
:102E4000202C03022E73C22CC38003A253B39232F0
:102E5000B392A6022E73022E73E53FB40B07D23253
:102E6000A232B392A622E53FB40B07C232A232B31C
:102E700092A62230081CC0E0787EE26013C3335073
:102E800005D0E0022ED412051550F6D0E0022E92A5
:102E9000D0E0E540604C24F84005E540022EEDE529
:102EA00040B40904A209803DB40A04A20B8036B4E0
:102EB0000C03D38030B40D0B303503022F0AD2350A
:102EC000D38022B40E04A20A801BB40F04A2778020
:102ED00014022F0AB40D06203503022F0AC235C38F
:102EE0008003A253B39237B39280022F0A022F0AB3
:102EF000E540B40B07D237A237B3928022E540B445
:102F00000B07C237A237B392802222C0F075F0FAC5
:102F1000D5F0FD75F064D5F0FDD0F022122F0B1224
:102F20002F0B122F0B122F0B122F0B122F0B2275A0
:102F30006908A2E7B392B4C293122F0BC2B4D29322
:102F4000122F0BC0E0E430B201040030B2010400E3
:102F500030B20104D36003D5E001C3D0E033D569BA
:102F6000D122D293C2B4D2B2122F0BC293122F1C11
:102F7000D293122F1C204C06201E0330722B788C0B
:102F80007601087480F608A2A3B392E4304C027470
:102F9000B3F6748008304C0274B0F608304C0274FA
:102FA00080F608F608F6022FEC788C760308768017
:102FB000087480A26692E5A2A3B392E4201E0B20BF
:102FC0007208A26992E1A23092E0F6087480201E95
:102FD0001220720FE55A54074480A26892E5A2A11C
:102FE000B392E4F6087480F608F608F675F00778F0
:102FF0008C7E007F00E62EFEE6122F2FF62FFF08B4
:10300000D5F0F2EED333122F2FF8EFD3336870627E
:10301000788CB6FF5D056BE56B24FE5014756B0272
:1030200020200ED2207518C0751900751A031216CB
:10303000AC204C06201E033072030230C77892E6A3
:1030400020E35720E24720E17E788DE6B60078083D
:10305000B64274D277757B037518B0751900751A6E
:10306000001216AC7518C0751900751A071216AC47
:103070008055E56B6014D56B1130200EC220751899
:10308000C0751900751A041216AC0230C7788D8607
:103090004208D26279A07A048008788DD26179944E
:1030A0007A05D27175F00FE6C4540FF755F0F5F0BC
:1030B00009E6540FF755F0F5F00908DAEAE5F0B43F
:1030C0000F051977EEC261D293C2B475F0051204F0
:1030D000E120B2061204E130B203D5F0F122D2931E
:1030E000C2B4D2B2122F0BC293122F1CD293122F42
:1030F0001C201E1F307123788C7611748008F6080E
:10310000A2A3B392E4F6748008F608F608F608F66F
:10311000023160788C761502311E788C7613087631
:1031200080087480A26692E5A2A3B392E420711194
:10313000A26792E1A2A4B392E0A26992E1A23092C6
:10314000E0F608748020710FE55A54074480A268A5
:1031500092E5A2A1B392E4F6087480F608F608F6A8
:1031600075F007788C7E007F00E62EFEE6122F2F8A
:10317000F62FFF08D5F0F2EED333122F2FF8EFD34E
:1031800033687050788CB6FF4B056AE56A24FE50B0
:1031900014756A0220210ED2217518C075190075A8
:1031A0001A051216AC3071030232337892E620E32E
:1031B0005520E24520E138788DE6B6007608B64223
:1031C00072D277757B037518C0751900751A0712CE
:1031D00016AC805FE56A6014D56A1130210EC221F9
:1031E0007518C0751900751A061216AC023233D262
:1031F00072788D8645D254803A788D864208D262A4
:1032000079A07A048008788DD26179947A05D27297
:1032100075F00FE6C4540FF755F0F5F009E6540FBA
:10322000F755F0F5F00908DAEAE5F0B40F0519777B
:10323000EEC261D293C2B475F0051204E120B20669
:103240001204E130B203D5F0F11204E12275F0036B
:103250001204C9D5F0FA1230DE75F0031204C9D594
:10326000F0FA122F6222204C0F30710C7518B075D5
:103270001900751A001216AC227005756E1E8002B8
:10328000D21922C298C29932201EF8309918C299D8
:10329000206005753400800EC0E0C0D075D01012DB
:1032A0003573D0D0D0E020980132C2982060FAC0A7
:1032B000D0C0E0E8C0E0305F05C25F754800E54F70
:1032C00024FE4003754F02E54820E712E548540705
:1032D00023246FC0E074003434C0E0E59922543FE9
:1032E00023232462C0E074003433C0E0E599221542
:1032F0006D023461023461D56DFAB54E08D20F7596
:10330000480002346702347FB462FA023461023446
:1033100061B42AF1023461F56D24C6E56D40E624FE
:10332000F5E56D50E0056D0234617820F2156D020F
:1033300034617821F2156D0234617822F2156D0244
:1033400034617823F2156D0234617824F2156D0230
:1033500034617825F2156D0234617826F2156D021C
:103360003461023495000233080002330E00023348
:103370001100023317000232EF000232EF00023276
:10338000EF000232EF0002332A0002333200023330
:103390003A000233420002334A0002335200023341
:1033A0005A000232F7000232F7000232F70002320E
:1033B000F7000232F7000232F7000232F700023261
:1033C000F7000232F7000232F7000232F700023251
:1033D000F7000232F7000232F7000232F700023241
:1033E000F7000232F7000232F7000232F700023231
:1033F000F7000232F7000232F7000232F700023221
:10340000F7000232F7000232F7000232F700023210
:10341000F7000232F7000232F7000232F700023200
:10342000F7000232F7000232F7000232F7000232F0
:10343000F7000232F7000232F7000232F7000232E0
:10344000F7000232F7000232F7000232F7000232D0
:10345000F7000232F7000232F7000232F7000234BE
:10346000950548254EF54ED0E0F8D0E0D0D032801A
:103470000E802A802D8030803280348040803EB49F
:103480000908754E0075480080D7B44208754E0093
:1034900075488080CC754E0075480080CAB51EDF27
:1034A00080BFB51FDA80BAF54980B6F54A80B2B55B
:1034B0004ECD754F201234BF75480080AA80D68546
:1034C0004936125E2ED260E536B44603023F18B488
:1034D0004704125E4422B4500D854A35125E09C27B
:1034E000ACC260D21722B45311854A35E54A70093F
:1034F000125E09C2ACC260D21222B4540D854A35A4
:10350000125E09C2ACC260D21122B4550D854A3593
:10351000125E09C2ACC260D21322B4560D854A3580
:10352000125E09C2ACC260D21422B4570D854A356E
:10353000125E09C2ACC260D21522B4580D854A355C
:10354000125E09C2ACC260D21622B44E12854A3550
:10355000E54AB4000A125E09C2ACC260D218222445
:10356000BF24E64004854A3522C26022C53725378C
:10357000C53722E53424F0400EE534232492C0E020
:1035800074003435C0E022759906C260753400D2EB
:10359000B6228036803B803D803F80408045804D14
:1035A000804F8058805680548052804D8057800DC7
:1035B0008015753403F59912356C053422A835E66B
:1035C00030002CE20235EF0236417537007403807B
:1035D000E4E51E80E0E51F80DC02368FE5377534B8
:1035E0000F80D21216EA123279883580C8E535800C
:1035F000C1E535A25392E080B9753403A83505358D
:10360000E676FF80B0E535C313603214700BA22D4F
:1036100092E0B392E1440480D614700BA22E92E0A3
:10362000B392E1440880C8147008A22F92E0440CC1
:1036300080BD147008A23692E0440C80B274FC8005
:10364000AEE5351470107408A26C92E0A26D92E1A0
:10365000A23092E280991470147410A22D92E0A20C
:103660002E92E1A22F92E2A23692E3808214700D94
:103670007418A22092E0A22192E10235EF14700B9F
:10368000A26E92E0A26F92E10235EFE40235EFE51F
:1036900036B441067534040235B5B4422AE53560C6
:1036A0000330191B53610F53620FC2AFE562B5615E
:1036B00006D2AFD30236BF056253620FD2AFC375D5
:1036C0006E1E74420235B2B444552008F7E535C386
:1036D000137022B3926A122C204040203C3D303DB2
:1036E0000B205205306A348003206A2FA26A92535D
:1036F000925202371B926A14C0E0030303540F2452
:1037000043F8D0E0540704FA7400D333DAFD306A8A
:1037100005FAE24A8004F4FAE25AF6E53680A5B4E6
:103720004B0280030237B4E53554F8B40812E5358E
:103730005407603714604314604714605C02358797
:10374000B4200FE5355407605914605C14605F02C3
:103750003587B42813E535A2E09253757A015003FA
:10376000757A02E5360235B2023587751AF4C26DF4
:10377000C26C755601755701805E751AF3D26D8063
:10378000EF751AF2D26CC26D755601755701C230D1
:10379000A230B392A7D26B803F751AF1D26CC26D82
:1037A0008031C26EC26F8039D26EC26F8033C26EFA
:1037B000D26F802DB4430FB53503755003753407B0
:1037C0007535A80235B5B44A20E5357019206D1657
:1037D000751AF0C20A1223AE75181075190F121659
:1037E000ACE5360235B2023587B4450675340602BB
:1037F00035B5B4510675340C0235B5B44D0EE5350A
:10380000121732E5365002B2E70236C4B44C0675E0
:10381000340E0235B5B4460280C9B4470280C4B440
:103820004F08C256C257C25880B9B45908C2007571
:10383000340D0235B5B45A08D20075340D0235B5D1
:10384000023587E570C2756002D275E55BF55CC232
:10385000592061093062030238AD023CD91205CD0E
:103860001220A7121F347028206E08206F1F123DEF
:103870004D501AC082C0831205A61222BCD083D03C
:103880008230620CE5426008121D9370030239B564
:1038900075543CD5501475183075190085501A129E
:1038A00016AC755003D2577553B4023CC41205CD03
:1038B000E54260F6B40206124D32023CD92071197D
:1038C000201D03303E13B4051078A0B60A0B08B6CD
:1038D00001028008B60302800302397808E675F019
:1038E0000AA4082675F00AA40826C5F0703B78A142
:1038F000B60339201D09C0F0123D08D0F0502A85CA
:10390000F05B85F05C12059C201D0F7518C07519C1
:1039100003855B1A1216AC023CD97518C0751902E2
:10392000855B1A1216AC023CD9023CBC201D09C0B2
:10393000F0123CF4D0F050F185F05B201D0E7518AC
:10394000C0751906855B1A1216AC800C7518C07507
:103950001905855B1A1216AC125438123D3AD2A2E0
:10396000C269C2A1D2681205A612234AA26172627C
:103970005003023851023CD912200A7035206E08DB
:10398000206F32123D4D502D1205A6C082C0831209
:10399000234AD083D082306119C082C0831205CD02
:1039A0001220A7D083D0827894797C7A05121CE407
:1039B0006003023890755400755003C258C25720F6
:1039C0005902C256C082C083123DF4D083D08250C7
:1039D00006123C78023CD9C082C083120A19D083F7
:1039E000D0825006123C78023CD9E58224CEE58391
:1039F00034FF5013123D3B400E122C205006123C57
:103A000069023CD9023BB912246F5012123C690280
:103A10003B70123C63023B70123C5D023B70206DB8
:103A2000F13039032053F1E5416058E54160092345
:103A30001205154003023A41023A83123C57023BF9
:103A4000703008F7301CF4304BF1A271304D01B3E7
:103A5000503130081BC0E0787CE26012C333500460
:103A6000D0E080D712051550F7D0E0023A70D0E0D0
:103A7000C082C083125CB8D083D0825006123C6EE4
:103A8000023B70301C49125C64A2E0921AA2E192DF
:103A90001BA271304D01B39205B4000520052280B0
:103AA0002BB4012220051A7518C0751900751A0962
:103AB0001216AC204706123C73023B70123CEA809F
:103AC0000E125BE18009B402ED2005DB125C0A30C6
:103AD000087930081CC0E0787BE26013C3335005DE
:103AE000D0E0023B4B12051550F6D0E0023AF1D07F
:103AF000E0207516A2719274858371858272123CE2
:103B0000E61205B7757002023CD9757000E5836551
:103B100071F5F0E582657245F07006123C7D023B5E
:103B2000707518C0751900751A0C1216AC30740C2B
:103B30007518B0751900751A001216AC123CA275F2
:103B4000181085711985721A1216ACC2A2C26912B8
:103B50003CE2A271920AD2091223AE123266123CE2
:103B6000A275181085831985821A1216AC12059C4D
:103B7000123D445003023CD9122C2040F8D2A3C27B
:103B800066C2A1D268D2A4C267755A0012324D1221
:103B90001E0DC082C08312234AD083D082206106CA
:103BA000206211023CD97894797C7A05121CE46079
:103BB00008023CC4121D9370F8301C24E4A21A922F
:103BC000E0A21B92E1B40305125C368013B4020537
:103BD000125BE1800BB40105125C0A8003125BB832
:103BE00030081CC0E07879E26013C3335005D0E0A0
:103BF000023CC412051550F6D0E0023BFFD0E03085
:103C00004E0FE58245836009023C11123C51023C93
:103C1000D9B25312326630531A75187085831985DC
:103C2000821A1216ACC2A3C266D2A1C268D2A4C2C2
:103C300067801875186085831985821A1216ACD2B0
:103C4000A3C266D2A1C268C2A4C26712059C023C8C
:103C5000D9125742023C80125742023C801257420E
:103C6000023C80125742023C801257428012125787
:103C700042800D1257428008125742800312574269
:103C80007570007571FF7572FF122CCE1232667559
:103C9000182085831985821A1216AC120589122CF8
:103CA000D822207116E55B04601114656F600C75F5
:103CB00018C0751901855B1A1216AC2212574212F0
:103CC00005788015125742122CCE120578122CD886
:103CD0007570007571FF7572FFC262C261E55CF5B7
:103CE0005B22125742221257422212574275F0327B
:103CF0001205E9227408F9747CF8752F01753003F8
:103D000075319812087B80127408F9747CF8752F4D
:103D10000175300375319012087B7881E6085608EA
:103D2000560460141205A61222BC306209E54260F6
:103D300005121D936002C322D32222E582249CE552
:103D40008334FF22E582249CE58334FF22A250E5E0
:103D50008245836010E582249CE58334FF5004A2F1
:103D60004F8002A25122E5822582F582E5833583C8
:103D7000F583E5822582F582E5833583F583E58247
:103D80002400F582E583345BF5837404F97400F84C
:103D9000752F01858330858231120856227881E69D
:103DA00054C0F5837882E630E402240A2323543C8D
:103DB0004583F5837881E6C4540375F00AA4F5F0D1
:103DC000E6540F25F0030303F5F053F0E085F0828D
:103DD00054034583F5837880E6C4540375F00AA440
:103DE000F5F0E6540F25F04582F58222C39582E571
:103DF000F0958322123D667800E2B4FF03023E7420
:103E0000126203123D9D787CA68308A6827800E2A8
:103E1000F58308E2F58208E2F5F008E2123DEC5085
:103E20002B7800E2F58308E2F582787C86F008E6DC
:103E3000123DEC50417802E2F58308E2F582787C8D
:103E400086F008E6123DEC402D023E747800E2F563
:103E50008308E2F582787C86F008E6123DEC401695
:103E60007802E2F58308E2F582787C86F008E612B3
:103E70003DEC5002C322D322C5372537C53722E592
:103E80005424E94008D2A3C266D2A2C2693098EF96
:103E9000C298E599123E78223099FDC299F599129F
:103EA0003E7822C2A3C266C2A2C269C2B6753700FA
:103EB0007405123E98E51E123E98E51F123E9822A8
:103EC0001204F91204F91204F9123EA3E536123E67
:103ED00098E537123E983099FD22120D72023EE3AA
:103EE000120D0EC0E0123EA3E536123E98D0E0124D
:103EF0003E98E537123E983099FD221204F9123EA1
:103F0000A3E536123E98797CE7123E9809DDF9E583
:103F100037123E983099FD22751A00755419D21E39
:103F2000E53E600B54F87007C231A231B392A5E5AB
:103F30003F600B54F87007C232A232B392A6D2A0EF
:103F4000C28EC28CC2ADC2ABC2ACC2AF7581CD90C5
:103F50003F5AC082C08375D00032D2AFD28C125E7D
:103F600009C2ACD299123EC0B2B5755419D29802AA
:103F70003F97B40922F537123E7FB51E27123E7FC8
:103F8000B51F21123E7FB4461B123E7FAF37123E53
:103F90007F6F7010123EC0D2B6D2A3C266D2A2C248
:103FA00069123E7FB40ACBF537123E7FB51EF5127B
:103FB0003E7FB51FEF123E7FF536B46D03024047DA
:103FC000B46E03024060B46F03024097B470030202
:103FD00040E4B471030240F8B47303024109B474BD
:103FE0000302410BB4750302411FB476030241374B
:103FF000B4770302414BB4780302415FB479030202
:104000004180B47A0302419CB46C030241B0B46BAA
:10401000030241D2B46A0302420DB4690302422989
:10402000B4680302426BB46703024283B4660302BE
:10403000429EB46503024362B46403024ADAB46187
:1040400003024B35023F97AF37123E7F6F70F51278
:104050003EC0D2B675F01E1204C9D5F0FA025FA3B5
:10406000123E7FFD1424E0402B123E7F2400FC7B97
:1040700000123E7FFEAF37123E7F6F70178EF0ED5D
:10408000F9747CF88B2F8C3085F03112087B123E4E
:10409000FB755419023F97123E7FFD1454E070F4F3
:1040A000123E7F2400FC247140EA7B02123E7FFE18
:1040B000EDFA787C123E7FF608DAF9AF37123E7FD0
:1040C0006F70D1C2A3C266C2A2C2698EF0EDF9744C
:1040D0007CF88B2F8C3085F0311207D0123EC975D9
:1040E000541980B0AF37123E7F6F70A8120B301298
:1040F0003EC0755419023F97AF37123E7F6F70096B
:10410000123EE0755419023F978089123E7FFD14DC
:1041100024E04048123E7F2400FC7B0102407112E3
:104120003E7FFD1454E07034123E7F2400FC2425B1
:10413000402A7B030240ACAF37123E7F6F701D02F6
:10414000415C123EC9755419023F97AF37123E7F4A
:104150006F7009123EDA755419023F970240947944
:10416000207D07123E7FF309DDFCAF37123E7F6FE3
:1041700070EA12531740E51261E4123EC9023F97FC
:10418000AF37123E7F6F70D41262031204F9123EF1
:10419000A3E536123E98121541023F97AF37123E03
:1041A0007F6F7066121163123EC0755419023F97FB
:1041B000123E7FFE123E7FFD123E7FFCAF37123E65
:1041C0007F6F7046120A964041123EC07554190224
:1041D0003F97123E7FFE123E7FFDAF37123E7F6F4C
:1041E0007028120A671204F91204F9123EA3E53688
:1041F000123E98EE123E98ED123E98EC123E98E573
:1042000037123E983099FD023F97024094AF371223
:104210003E7F6F70F51204F91204F9123EA3E536E1
:10422000123E981215D1023F97AF37123E7F6F7042
:10423000D9120D0660027401C0E0120D6A600274AA
:1042400002D0F045F0700A120B7B1219291211638B
:10425000E4C0E0123EA3E536123E98D0E0123E984C
:10426000E537123E983099FD023F97123E7FFD14CC
:1042700054E07027123E7F2400FC2471401D7B0017
:104280000240AC123E7FFD1454E0700F123E7F24BA
:1042900000FC242540057B010240AC024094AF376E
:1042A000123E7F6F70F51204F91204F9123EA3E575
:1042B00036123E987401123E98744E123E98746EF7
:1042C000123E987448123E987437123E9874001249
:1042D0003E98748D123E987420123E9874DA123E05
:1042E000987400123E98740F123E9874A0123E9873
:1042F0007480123E987400123E987400123E9874B6
:1043000020123E987400123E987400123E98740079
:10431000123E987400123E987400123E9874001277
:104320003E987400123E987400123E987400123E3B
:10433000987400123E987400123E987400123E98D1
:104340007400123E987400123E987400123E9874E5
:1043500000123E98E537123E983099FD023F9702D1
:104360004094123E7FF583123E7FF5822460E58300
:1043700034F040EB12464B123E7FFD1454E070DFE8
:104380007800123E7FF208DDF9AF37123E7F6F7082
:10439000CE123EC075F0051204C9D5F0FA123EC91E
:1043A000751A013008B93007B61246BF1246A51279
:1043B0004659121E0D789479007A0A75F00FE3546D
:1043C0000FF652F00809DAF643F0F0E5F0047894BD
:1043D000797C7A05121CE4600B12447A5006751A37
:1043E0000402435F1246A5124659121E0D78A079A9
:1043F0000A7A0675F00FE3540FF652F00809DAF660
:1044000043F0F0E5F00478A079817A03121CE460AF
:104410000B1245185006751A0602435F1246A51284
:104420004708751A65023F97C0E07830E583F208C7
:10443000E582F2D0E022C0E07832E583F208E5823E
:10444000F2D0E022C0E07830E2F58308E2F582D0D5
:10445000E022C0E07832E2F58308E2F582D0E02283
:10446000E5822400F582E583341BF58322E582246E
:1044700000F582E583343BF58322124659AB83ACC9
:1044800082901B00C0837900752F038583307531BE
:10449000009000361207851208F61207851209549B
:1044A0009000367A80E0A3F5F0E0A36C7005E5F0AB
:1044B0006B6017DAF0D0830583740024C0E5833481
:1044C000C550C174051245C7D322D083EA2AF5F03E
:1044D000E4C395F0F582124428789479007A0A753D
:1044E000F00FE3540FF652F00809DAF643F0F0E566
:1044F000F004600C121F39700A74061245C7D322EB
:10450000121F39E5822582F582E5833583F5831212
:1045100044601244360248DF124659AB83AC8290A5
:104520003B00C0837900752F03858330753100907F
:1045300000361207851208F61207851209549000FA
:10454000367A80E0A3F5F0E0A36C7005E5F06B60CF
:1045500017DAF0D0830583740024C0E58334A550B6
:10456000C174051245C7D322D083EA2AF5F0E4C30B
:1045700095F0F58212442878A0790A7A0675F00F32
:10458000E3540FF652F00809DAF643F0F0E5F004D0
:10459000601D12201A701BAB83AC82124659EBB51A
:1045A0008306ECB58202C32274041245C7D32212DB
:1045B000201AE5822582F582E5833583F58312444E
:1045C0006D1244360248DFF51A22C082C083E583AB
:1045D000125316D083D082C082C083E58212531654
:1045E000D083D08222C082C0837F00E58224F0C0C5
:1045F000E0E58334D8C0E05007D083D0820F80EB51
:10460000D0E0D0E07F00E5822418C0E0E58334FCF0
:10461000C0E05007D083D0820F80EBD0E0D0E07FA5
:1046200000E582249CC0E0E58334FFC0E05007D061
:1046300083D0820F80EBD0E0D0E0E58275F00A8471
:10464000C0F0F5F0D0F0D083D08222C0E07834E51D
:1046500083F208E582F2D0E022C0E07834E2F5830C
:1046600008E2F582D0E0227881E61253167882E6DD
:104670001253167883E612531678A0E61253167872
:10468000A1E612531678A2E612531678A3E6125347
:104690001678A4E612531678A5E6125316120E04E5
:1046A00022120E04227400123E987400123E987476
:1046B00000123E987400123E987400123E982275C3
:1046C000831B75821B75F040C0F0C082C083752FBC
:1046D000018583307531001207851208F6D083D02A
:1046E00082C082C083752F03858230753100120726
:1046F000851209BCD083D08205830582D0F0D5F025
:10470000C77532FF7533FF227401F97418F8752FDD
:104710000075300075310012087B7401F97419F8C6
:10472000752F017530D97531FF12087BAC18124610
:1047300059E5822420F582E583347DF583C082C06B
:10474000837401F97441F8752F00858330858231B7
:1047500012087BD083D0827401F97410F8752F0091
:1047600085833085823112079F7810E2F5F0E518D5
:104770002541C395F0F518124659E58275F008A455
:104780002420F582500205F0A8F0E58375F008A416
:10479000282400F5837408F9747CF8752F0085834C
:1047A0003085823112087B787CE5187A082608DA91
:1047B000FCF518789479007A0A75F00FE3540FF637
:1047C00052F00809DAF643F0F0E5F00412522578C9
:1047D000A0790A7A0675F00FE3540FF652F0080933
:1047E000DAF643F0F0E5F00412522D7408F9747C07
:1047F000F8752F008583308582311207D0787CE5EB
:10480000187A08C39608DAFBF518124659C3E582F0
:1048100033F582E58333F583C3E58233F582E5839F
:1048200033F583E5822400F582E583245BF583C0BC
:1048300082C0837404F9747CF8752F0185833085F8
:10484000823112087BD083D0827404F97412F87517
:104850002F0185833085823112079F787C7912E59C
:10486000197A0426F5F0E3C5F0C395F00809DAF3E8
:10487000F5197401F97418F8752F00753000753149
:10488000001207D07401F97419F8752F017530D929
:104890007531FF1207D075831B75821B75F040C000
:1048A000F0C082C083752F038583307531001207F5
:1048B000851208F6D083D082C082C083752F01850F
:1048C00082307531001207851209BCD083D0820571
:1048D000830582D0F0D5F0C77532FF7533FF221201
:1048E0004452E5828583F0124444C39582C0E0E5DA
:1048F000F09583D0F045F07002C32250030249FACC
:10490000124452C0E0C3E58224FEF582E58334FF01
:10491000F583D0E0124436E5828583F0124444B535
:104920008207E5F0B58302C322124444AF831244E8
:1049300052EFB58310AE82900034787CE0F6A30885
:10494000E0F602495D7EFE8F8305837402F9747C74
:10495000F8752F0385833075310012087B79007557
:104960002F038F307531009000361207851208F63C
:104970001207851209548F837582001244447D000A
:10498000E5836F7002AD82ED2436F58275830050A9
:10499000020583C3EE9D20E05A03FCC082C083A3BE
:1049A000A3E0FAA3E0FBD083D082EAF0A3EBF0A36C
:1049B000DCE9EE2436F58275830050020583787CAD
:1049C000E6F0A308E6F07900752F038F307531000B
:1049D0009000361207851209A81207851209BC85B6
:1049E0002F32853033124452EFB58303024ACE0F83
:1049F00002492E74081245C7D322124444AF8312D1
:104A00004452EFB58310AE82900034787CE0F6A378
:104A100008E0F6024A2E7E008F8315837402F97433
:104A20007CF8752F038583307531FE12087B790081
:104A3000752F038F307531009000361207851208EC
:104A4000F61207851209541244447DFEE5836F7007
:104A500002AD82ED2436F58275830050020583C3D2
:104A6000ED9E20E06B03FCC0E0C3E58224FEF582EE
:104A7000E58334FFF583D0E0C082C083E0FAA3E091
:104A8000FBA3EAF0A3EBF0D083D082DCDAEE24368D
:104A9000F58275830050020583787CE6F0A308E672
:104AA000F07900752F038F307531009000361207B2
:104AB000851209A81207851209BC852F328530336B
:104AC000124452EFB58303024ACE1F0249FFC322AC
:104AD00074091245C7D322024094123E7FF5831217
:104AE0003E7FF582AF37123E7F6F70EBC01EC01F56
:104AF00085831E85821F121C697401F9747CF87508
:104B00002F0075300075310012087B787CE6C39564
:104B10001EC3951FD01FD01E251E251FF67401F938
:104B2000747CF8752F007530007531001207D012B3
:104B30003EC0023F97123E7FF583AF37123E7F6F34
:104B400070951204F91204F91204F9123EA3E53625
:104B5000123E987400123E98E51A123E98740012A4
:104B60003E987400123E987400123E987400123EF3
:104B700098E537123E983099FD023F97904B84C0DC
:104B800082C083327581CD75D000025FA3C082C020
:104B900083E5822420F582E583347DF5837401F971
:104BA0007441F8752F008583308582311207D0D08B
:104BB00083D082C082C083E58275F008A42420F5EA
:104BC00082500205F0A8F0E58375F008A4282400BF
:104BD000F5837404F9747CF8752F00858330858221
:104BE000311207D0A3A3A3A3747C2404F5F07404AA
:104BF000F9E5F0F8752F008583308582311207D0F2
:104C0000D083D082C20722120D0EC0E07401F97465
:104C10007CF8752F0075300075310012087B787CA8
:104C2000E6D0F0C395F0F67401F9747CF8752F00A6
:104C30007530007531001207D022120578C2AF809E
:104C4000FE30081CC0E07879E26013C3335005D011
:104C5000E0024CD812051550F6D0E0024C60D0E0CE
:104C6000D2A3C266C2A1D268D2A4C2671205A6129C
:104C7000234A206106206230024CD81205DF121F41
:104C8000347055123D444050206E08206F4C123D48
:104C90004D50471205A61222BC30623CE5426038F6
:104CA000121D937033024CDAE542602C1205DF12BC
:104CB000200A7024123D44401F206E08206F1B12F2
:104CC0003D4D50161205A612234A30610B78947997
:104CD0007C7A05121CE46002D322304E18E582452E
:104CE000836012E5416009231205154003024CF36D
:104CF000024CF580E3B253C312326630531A751872
:104D00007085831985821A1216ACC2A3C266D2A11D
:104D1000C268D2A4C267801875186085831985821D
:104D20001A1216ACD2A3C266D2A1C268C2A4C267CC
:104D3000C32278A0E6B40A1708E6B40545122C2071
:104D40004009124C41400412059C2212057822753C
:104D5000F00AA4F5F008E625F0B46326D2A3C266F3
:104D6000C2A2D269C2A1D268D2A4C267C0E01205B1
:104D7000A612234A900000121E0D20610920622B0A
:104D8000D0E0120578221205DF7894797C7A05123A
:104D90001CE470EC30503A1205A61222BC3062E0DE
:104DA0001205DF121D9370D8024DD11205DFE542C6
:104DB00060CE121D9370C93050171205A612234AF7
:104DC0003061BD1205DF7894797C7A05121CE4709D
:104DD000AF1205A6D0E0B40B081250964024024F43
:104DE0000BB40C081250D74019024F0BB40D081227
:104DF0005102400E024F0BB40E0B12511140030230
:104E00004F1A024F07B40F28126203125283401D3B
:104E1000F824DC4018E87880F6125283400FF8241A
:104E2000A0400AE8787FF61261E4024F0B024F07B8
:104E3000B410028003024EA71262031222B820545B
:104E4000061222B83054E6121703C0E0D0E0F8246E
:104E5000F640DAE8131354C07881F612528340CD3D
:104E600060CBF824ED40C6E87882F61252834034D5
:104E70006032F824CE402DE8788146F61222B82020
:104E800054061222B830541C121703C0E0D0E0F8C8
:104E900024F94010E813131354C0788246F61261C7
:104EA000E4024F0B024F07B4111512171BB4010C8B
:104EB00012171BB40706125120024F0B024F07B402
:104EC00013202038F712234A20620B3061EE121DA6
:104ED000B57034024C3AE542602D121DD1702802A3
:104EE0004C3AB4632212171BB40A1C12171BF57735
:104EF00090017D700390018A75F0641204C9D5F0A9
:104F0000FA024F0B024F0712057822124C07751850
:104F1000C0751900751A0A1216AC12059C2275414B
:104F200000787C75F00876FF08D5F0FA22EFC0E033
:104F3000C25A789979817A06EA30E004E60880025C
:104F4000E6C4540FFFEA30E004E7098002E7C454E6
:104F50000FB40F10BF0F10EA6406600B205A1ED06A
:104F6000E0FFE422BF0F06D0E0FF740122205AF7D1
:104F7000F5F08F476F6002D25ADABD80DFE5F0C3EB
:104F800095475002F4041460D6B408DB80D17894BD
:104F9000797C7A057401B6FF02800FB7FF02800AA0
:104FA000E66770060809DAF8E422740122124FB8A5
:104FB000E58245837001D3228005D0E002500912BA
:104FC000171BC0E024F640F2D0E075F00AA4F58289
:104FD0008005D0E002500912171BC0E024F640F211
:104FE000D0E0258275F00AA4F58285F0838005D093
:104FF000E002500912171BC0E024F640F2D0E02571
:1050000082F58250020583C322D322C082C08390DE
:105010000000121E69124F8E701AE5828583F0D04F
:1050200083D082B5821FC5F0B5831AC082C083F5D4
:105030008385F082A3E583B40FD8E582B4A0D3D0F2
:1050400083D082C322D322C082C083900000121E6C
:1050500069124F2D701AE5828583F0D083D082B516
:10506000821FC5F0B5831AC082C083F58385F082A4
:10507000A3E583B40FD8E582B4A0D3D083D082C394
:1050800022D32212234A306131125225121DE7C366
:10509000229000008008124FAD401F1205A6122377
:1050A0004A3061161205DF121E0D12522512500BE6
:1050B0004008754100124B8DC322D3221222BC300E
:1050C00062F8E54224FD24FC40F012522D121DFA34
:1050D000C3229000008008124FAD40DE1205A612D8
:1050E00022BC3062D5121E0D12522DE542600B24F7
:1050F000FD24FC40C512504740C0754100124B8D45
:10510000C322124FAD4008124F1E124B8DC322D343
:1051100022124FAD4008121E0D12516FB322D3223E
:10512000C20790002874D8F974FFF8752F018583A1
:1051300030858231120CBE75830175F01E752F000B
:10514000858330753100C0F0C083120785120C9E34
:10515000D0830583D0F0D5F0E4907D007420F974FD
:10516000FFF8752F01858330858231120CBE2278BD
:105170007CE6080808080856B4FF02D322C322754B
:105180001E30751F30C271C27275F005C0F0D2A317
:10519000C266C2A2D269D2A1C268D2A4C267124FAB
:1051A0001E12234AD0F0206109206206D5F0DD02EC
:1051B00051F6125245403F12059C7881E6B4FF0536
:1051C000C32275F005C0F012234AD0F0206206D544
:1051D000F0F30251F6E542B4021C78A0E624F64052
:1051E0001508E624F6400F78A0E62430F51E08E600
:1051F0002430F51FC322120578D3227546008003A0
:10520000754601C25512234A20620B30610A0546D9
:10521000E54624F550EFD322E5466007D255B40A9F
:10522000027400C3227894797C7A05800678A0798C
:10523000817A03E608540FC4F5F0E608540F45F0F0
:10524000F709DAEF22206131306236E54260062448
:10525000FD24FC402C12522D1205A675F005C0F05D
:10526000122346D0F0206111205406D5F0F00252EE
:1052700081121703B40B0A8003125225754100C333
:1052800022D3221222B82054061222B830542B12F4
:105290001703C0E0D0E0F824F6401F1222B82054D3
:1052A000061222B8305413121703C0E0D0E0F5F014
:1052B00024F64006E8C445F0C322D3221252CC752E
:1052C000F0641204C9D5F0FA12054B2275F03C12B5
:1052D00005E9C2A075F03C1205E9D2A075F01412E0
:1052E00005E9C2A075F03C1205E9D2A075F01412D0
:1052F00005E9C2A075F0141205E9D2A075F01412E8
:1053000005E9C2A075F0141205E9D2A02275F00AD1
:1053100084C0F0D0F022227825E254C07078E27583
:10532000F00A84C445F0787EF67824E254C07066B2
:10533000E275F00A84C445F0787FF67823E254E001
:105340007054E275F00A84C445F07880F67822E261
:10535000604454E07040E275F00A84C445F0C0E057
:105360007820E2030354C0D0F045F07881F678212C
:10537000E2602354F0701FE275F00A84C445F0C067
:10538000E07826E254F8700EE2C42354E0D0F045F1
:10539000F07882F6C322D32290000075F019C0F095
:1053A0007402F9747CF8752F01858330858231127F
:1053B000087B787DB6FF02800E18E55B300805B4E7
:1053C000FF02E56F666011E5822410F58250020548
:1053D00083D0F0D5F0C8C322D0F0A3D32230084D3B
:1053E000E58224FFF582E58334FFF58375F019E546
:1053F000822480E58334FE5005900000800AE58217
:105400002410F58250020583C0F07402F9747CF810
:10541000752F0185833085823112087B787DB6FF38
:1054200002800518E6B55B07D0F0D5F0C2C322D0E4
:10543000F0A3D32222025463300FFAC20F12531783
:1054400040F31261E40254667822E212530D78218F
:10545000E212530D7823E212530D7824E212530D19
:1054600002548A1262037881E6C45403E6540F782A
:1054700082E6C45401E6540F7880E6C4540FE65423
:105480000F787FE6C4540FE6540F30080A12539881
:105490005005125434800312549B22E55BB4FF067E
:1054A0009002CA0254DAB4000690010A0254DAB437
:1054B00010069001130254DAB4110690011C025434
:1054C000DAB420069001260254DAE55B75F06484B4
:1054D000C0F0D0E012530D90015222201C01227521
:1054E0008205125B48600F75F0021204C9D5F0FA0C
:1054F000D582EF125B4A747578431205FA50152075
:105500007614D276125B4A7518C0751900751A0D9B
:105510001216AC22C276126203203F0420402E22D3
:105520007880E6543FF5F0793FE365F0701C09E3BD
:10553000787F667015204111D241125B4A7518C000
:10554000751900751A0D1216AC2230402A7880E6C3
:10555000543FF5F07941E365F0701C09E3787F660C
:105560007015204111D241125B4A7518C07519009F
:10557000751A0D1216AC22C24122C2AC1216EA6094
:1055800024F51888191211D653610F53620FC2AF58
:10559000E562B56106D2AFD30255A3056253620F2F
:1055A000D2AFC380D7D2AC227E007F64900000755A
:1055B000F000E49325F0F5F0A3C3E5829EE5839F18
:1055C00040F0E5F0700122E5F0C0E0E583125316EB
:1055D000E582125316D0E0125316C2ADC2ACD21EF1
:1055E00012056320B7FA75F0C81204C9D5F0FA3075
:1055F000B7FD75F0C81204C9D5F0FA125E0922751C
:10560000F0641209CF20E51230E30F221204E1B258
:10561000B51204E1B2B5D5F0F322C2AFB2B51204AF
:10562000E1B2B51204E1D5F0D9C2A075F03212563C
:105630000CD2A075F03212560CC2A075F032125680
:105640000CD2A075F03212560C75F09612560C80E2
:10565000D82230083C7400785312060940337F0882
:105660007E00747878431205FACE13CE05E0DFF49D
:10567000201F0E740078631206095005EE655D6008
:10568000108E5D8E5B7518C0751904855B1A121635
:10569000AC22C2AF75181075190FF51A1216ACD2DC
:1056A000AF223008097401785312060950012274A0
:1056B0007778431205FAE492E0C0E07476784312FA
:1056C00005FAD0E033FE201F0E740178631206093C
:1056D0005005EE655E60D78E5EEE20E10630E02E6E
:1056E00002572B30E017A26D726C50C2C26DC26CB3
:1056F00075560175570174F812569280B1D26DC279
:105700006C75560175570174F712569280A0206C83
:105710009DD26CC26D755601755701C230A230B36F
:1057200092A7D26B74F61256928083A230826C409C
:10573000F8D26CC26DC20A1223AE74F512569202F0
:1057400056AEC082C083D083D082222222C2A075EE
:10575000F0141204C9D5F0FAD2A075F0141204C9DD
:10576000D5F0FA22C2A075F03C1204C9D5F0FAD2E5
:10577000A075F0141204C9D5F0FA2212574D125731
:105780004D12576412574D75F0641204C9D5F0FAE2
:105790002212576412574D12574D12574D75F0642F
:1057A0001204C9D5F0FA22305309C2A3C266D2A4AA
:1057B000C26722D2A3C266C2A4C26722300849309F
:1057C000081CC0E0787AE26013C3335005D0E002D1
:1057D00057F412051550F6D0E00257DED0E0D26E35
:1057E000201F032070227518C0751900751A0F123A
:1057F00016AC8014C26E201F0330700C7518C07573
:105800001900751A101216ACA26E9270220943008C
:10581000A00954009F0966009E0977009D09890030
:105820009C099B009B09AD009A09BF009909D20011
:105830009809E4009709F700960A0A00950A1D00E6
:10584000940A3000930A4300920A5700910A6B00B1
:10585000900A7F008F0A93008E0AA7008D0ABB0072
:105860008C0AD1008B0AE7008A0AFE00890B14001B
:10587000880B2B00870B4300860B5C00850B7500A3
:10588000840B8E00830BA700820BC100810BDB0011
:10589000800BF6007F0C10007E0C2B007D0C470067
:1058A0007C0C64007B0C81007A0C9E00790CBB00A0
:1058B000780CDB00770CFB00760D1B00750D3B00B0
:1058C000740D5B00730D7D00720D9F00710DC200A1
:1058D000700DE4006F0E07006E0E2C006D0E51006F
:1058E0006C0E76006B0E9B006A0EC100690EE9001B
:1058F000680F1100670F3900660F6100650F89009E
:10590000640FB300630FDE00621009006110340001
:1059100060105F005F7F4290580DE493A3F5F0E4C0
:1059200093A3C3958BE5F0958D5015A3A3DFEBE50D
:105930008224FFF582E58334FFF583E49314800B22
:10594000A3E493BF420590580D8010C0E0E5822487
:10595000F9F582E58334FFF583D0E02290003AE048
:10596000A28733F02290003B7400F090003A745507
:10597000F090003C74FFF090003E7405F090003D04
:105980007412F0D28122D286A2A4C0D0D2A475F023
:1059900000D5F0FDD5F0FDC28E53890F43891075F7
:1059A0008B00758D00C28FC2AFC2A4D28E20860339
:1059B000308FFAC28E308F06758BFF758DFFD2AF98
:1059C000D0D092A422F024FD4005308102C2812271
:1059D00090003EE0D5E0EE7442F0125986D281E5A7
:1059E0008B2499E58D34F24014E58B24E1E58D3468
:1059F000F3400EE58B249CE58D34FF400874158040
:105A000006741180027412FE90003DE06E6010EE8C
:105A1000F020030B7518C07519008E1A1216AC22EF
:105A200012595C603604603390003CE020E010D2F4
:105A3000E0F090003BE070047405F022E4F0229066
:105A4000003BE0602914F070252002227518C07513
:105A50001900751A141216AC025A6E90003CE03010
:105A6000E00DC2E0F090003BE070D1743CF0229079
:105A7000003BE060F914F070F52002F27518C07573
:105A80001900751A131216AC80E41259D0125A205C
:105A900022C2B61259861259157537007403123E88
:105AA00098E51E123E98E51F123E98744E123E98DD
:105AB000740C123E987400123E98740A123E98C0FC
:105AC00082C083A3A3A3E49375F064A4C0E0E5F0CF
:105AD000123E98D0E0123E98A3A3A3A3E49375F0DE
:105AE00064A4C0E0E5F0123E98D0E0123E98D08366
:105AF000D082E493123E98A3E493123E98A3A3A30A
:105B0000E493123E98A3E493123E98E58D123E98DA
:105B1000E58B123E98E537123E983099FD22120827
:105B2000C6C28474541208E0E41208A01208B3F547
:105B3000F06448256733F567E5F02568B2E003F5C2
:105B400068D9E9D284222222E4227583DD75F0101F
:105B5000752F03858330753100C083C0F01207852F
:105B6000120C9ED0F0D0830583D5F0E47532FF751A
:105B700033FF125B4722025BA9C082C08375820596
:105B8000C082125B48D082601CC2A075F00F120464
:105B9000C9D5F0FAD2A075F0051204C9D5F0FAD52E
:105BA00082DE125B4AD083D082E5822400C0E0E529
:105BB0008334DDF8D0E0C322125B79C082C083F564
:105BC000828883787C76007401F9747CF8752F03E1
:105BD0008583308582311207D0D083D082125B4713
:105BE00022125B79C082C083F5828883787C76023A
:105BF0007401F9747CF8752F038583308582311226
:105C000007D0D083D082125B4722125B79125B7976
:105C1000C082C083F5828883787C76017401F97430
:105C20007CF8752F038583308582311207D0D083AD
:105C3000D082125B4722125B79C082C083F58288D2
:105C400083787C76037401F9747CF8752F0385835F
:105C5000308582311207D0D083D082125B47221266
:105C60005B768003125B79C082C083F5828883747F
:105C700001F9747CF8752F03858330858231120811
:105C80007B787CE6B40102800CB402028007B40386
:105C90000280027400D083D082221208C6C28474AB
:105CA000541208E0E41208A01208B3B402057567A4
:105CB000018002D9F3D284227567007583DD75F007
:105CC0000F752F03858330753100C083C0F0120734
:105CD000851208F61207857900125C9AD0F0D083FD
:105CE0000583E5677026D5F0D8752F038583307559
:105CF00031001207851208F612078579A0125C9A06
:105D00007532FF7533FFE5677002D322C322C28C60
:105D1000758A45758C5DD28CB20120010132C0D0EC
:105D2000C0E0C0F075D008D265201E04E5556002C1
:105D3000B2B5121702125DEA051DE51D20E03920FB
:105D4000E136201E3A206905A230B392A2E51D304B
:105D5000E203122CE2E51D541F7013E4B55628B57A
:105D60005147B55356B56E5EB57B5FB55463E4B528
:105D70005545B5526AB54F6BD0F0D0E0D0D032E582
:105D80001D541F60E680F1304A0CE55724C24003E1
:105D9000D557CC75573CD556C6C209206CC1C23008
:105DA000A230B392A7D26B80B6D551B6C209755353
:105DB000B4D258D25B80AB155580B7D553A7C25625
:105DC000C257C258809F156E809ED57B9EC2778039
:105DD0009AD5549A755003301E03024B7C80861569
:105DE000528092D54F92D25F808EE51DA2E330663D
:105DF0000292A330690292A230680292A122C2B636
:105E0000206002D2B6125E093275C800C2ADC2ACC3
:105E100075CBFF75CA9875CDFF75CC98759853C230
:105E200098C299D2ACC2BC75C8347599062275C89F
:105E300000C2ACC2AD75980075CC2B75CDEBD2AD60
:105E400075C8042275C800C2ACC2AD759800E58A59
:105E5000242BF5CC540F658C24EBF5CDD2AD75C851
:105E600004227580FF7590FF75A0FF758F011209E0
:105E7000DCD21ED2A0755600755700C230A230B3D6
:105E800092A7C231A231B392A5C232A232B392A676
:105E9000E4F541784375F010F2D5F0FCC26CC26DA8
:105EA000C26EC26FC22DC22EC22FC236C254C2569B
:105EB000C257C258755301755400C25BD25FC260AD
:105EC000D265C217C211C212C213C214C241C21596
:105ED000C216756C01C220C221754F10E4F548F559
:105EE00049F54AF534F536751E00751F80753E0775
:105EF000753F00E4F551F559F558F561F562F54443
:105F000075430F75450F751D0474377836F2783771
:105F1000F27838F2D227D228D229D234743778399D
:105F2000F275500375520178A87A0576FF08DAFBFE
:105F3000C20F7820E47A07F208DAFCC210755BFF22
:105F4000855B5DC219C208C243756E1E757000C2C2
:105F500075C20DC20EC209C20AC20BC271C2721250
:105F600018737555FAB2B57532FF7533FF75770042
:105F7000D276757A00782F740AF2D204125965C26B
:105F800077757B01758901758A3E758C5DC2B9D2C2
:105F9000A9D28CD2B6125E09D2AFD293C2B4D2B219
:105FA000B2B522C21E755A0375F0031204C9D5F0AA
:105FB000FAC271C2721230DE755A0375F003120410
:105FC000C9D5F0FAC271C272122F62C2AF020000CC
:105FD000D6435243206C696E6961203300D7435227
:105FE00044206C696E6961203400C2AF7555FAB205
:105FF000B51204E1B2B51204E1B2B5D2A07581CDFB
:1060000075D000125E621257421255A8125B4A12F6
:1060100020BF7555FA1210D4755A0312324D12056D
:10602000B0751880751904751A6E1216ACD21F302F
:10603000080F120F6C1256521256A21254DB12574E
:10604000BCD2B7D2AFC21EC21F00000020B70912D7
:1060500004E120B7030220D9300815304303120FA2
:106060006C30080C1256521256A21254DB1257BC56
:10607000E5706003D57008125A8A125438800CD229
:10608000A3C266C2A1D268D2A4C267E56E70063010
:10609000420312557AC269D2A1C2681257A7C271CF
:1060A000C272D26B12234A2062052061028017302F
:1060B0003A093057061257420260BE123843782F11
:1060C000E215E0F27008782F7414F20260418091BA
:1060D0000074A2126165E81261A0E91261A0126168
:1060E000D72274A2126165E81261A0E71261A009CB
:1060F000D582F81261D72274A2126165E81261A0FC
:1061000074A31261651261C0F709D582041261D7C8
:1061100022C296D297000000C29780E974A2126151
:1061200065E81261A01261292274A31261651261EF
:10613000C0F91261D72274A27A08C296000000C288
:1061400097335005D29602614BC296D29700000059
:10615000C297DAEDD29600D297000000309604C2C2
:1061600097C322D3227A08D296D29700000000006B
:106170000000000000000000000000C296000000C7
:10618000C297335005D29602618CC296D297000016
:1061900000C297DAEDD29600D297000000C2972293
:1061A0007A08335005D2960261ACC296D2970000AD
:1061B00000C297DAEDD29600D297000000C2972273
:1061C0007A08D296C29700000000D297C330960199
:1061D000B333DAF0C29722C296000000D2970000D3
:1061E00000D29622787C76000876007880E6543FCC
:1061F000F67800797CC0827582071260E2D0821244
:1062000004C9227802797EC0827582051260F7D0B7
:1062100082227882E603C4540775F018A4C0E0789F
:1062200080E6C4540375F00AA4F5F0E6540F25F097
:10623000D0F025F075F03CA4C0F0C0E0787FE6C453
:10624000540775F00AA4F5F0E6540F25F0D0F025B8
:10625000F0F5F0D0E03400C5F022000000000000AE
:10626000000000000000000000000000000000002E
:10627000000000000000000000000000000000001E
:10628000000000000000000000000000000000000E
:1062900000000000000000000000000000000000FE
:1062A00000000000000000000000000000000000EE
:1062B00000000000000000000000000000000000DE
:1062C00000000000000000000000000000000000CE
:1062D00000000000000000000000000000000000BE
:1062E00000000000000000000000000000000000AE
:1062F000000000000000000000000000000000009E
:10630000000000000000000000000000000000008D
:10631000000000000000000000000000000000007D
:10632000000000000000000000000000000000006D
:10633000000000000000000000000000000000005D
:10634000000000000000000000000000000000004D
:10635000000000000000000000000000000000003D
:10636000000000000000000000000000000000002D
:10637000000000000000000000000000000000001D
:10638000000000000000000000000000000000000D
:1063900000000000000000000000000000000000FD
:1063A00000000000000000000000000000000000ED
:1063B00000000000000000000000000000000000DD
:1063C000000000000000000000000000000050522B
:1063D000343032207665722E3131302E37204864C9
:1063E000773A482034303030752032382D30362D11
:1063F00030342031303A343120204352433D003F85
:00000001FF
:0300000306028072
